:020000000528D1
:1000080025288B138B1B0528831607308500E030C5
:10001800860047308100831200308500003086005A
:100028000B108B160C3084008001840A4F300402B8
:10003800031D1828F030810005128B175B2064001F
:1000480023289100030892000B193E208B183B20AF
:100058000C0833210D0833210E0833210F10120824
:100068008300110809008B138B1B372808008B109D
:100078000B1208000B11D9308100080057200030FE
:100088009F000130A200253084000C14A9200C1216
:10009800B7205520080025089E0000309F009720B3
:1000A80008008B1708008B138B1B572808000516B0
:1000B8008E3069200030692005121C210516803019
:1000C80069200030692005120800A0008316051178
:1000D80083120830A1006400A00C031C75280515C4
:1000E800762805111C2185151C218511A10B6F2867
:1000F800831605158312051585151C218511080021
:100108008316051583120830A100640085151C218B
:10011800051990280310912803149D0C85111C21A2
:10012800A10B8928080005309C000C10A9200C148C
:10013800A9200C16B7201D081E020319A7289C0B1E
:1001480099280E1708000E130800C720A030D120E8
:100158001F08D1200C18B2281E08D12010210C1C11
:1001680022210C100800C720A130D120EC200C1A45
:10017800C2281D088000840AA20BC52810210C166D
:100188000800FF20BA288316051183128515051566
:100198001C2105111C2185110800A00083160511DA
:1001A80083120830A1006400A00D031CDD2805158A
:1001B800DE2805111C2185151C218511A10BD728C6
:1001C800831605158312051585151C218511080050
:1001D8008316051583120830A100640085151C21BB
:1001E8000519F8280310F92803149D0D85111C2101
:1001F800A10BF128080083160511831205111C2193
:1002080085151C2185111C210800831605118312F0
:10021800051585151C2185118316051183120511F5
:100228001C2185151C210515831605158312080048
:100238000A3093006400930B1E29080006309300CF
:1002480064009308031D24290800193093002E29FF
:10025800C830930064009308031D2E290800A400E9
:100268000830A300061000000614A40D031C061095
:1002780000000000000006100000A30B3829240825
:0202880008006C
:1007C0004734503443345F34343441343434203487
:1007D0003034563430343134203400342834433407
:1007E0002934203450344D344234203432343034BF
:0607F00030343234003405
:00000001FF
